:020000040800F2
:100000004804002009010008D3190008D519000888
:10001000D9190008DD190008E119000800000000E6
:10002000000000000000000000000000E7190008C8
:10003000E519000800000000E9190008EB190008A4
:100040002301000823010008230100082301000800
:1000500023010008230100082301000823010008F0
:1000600023010008230100082301000823010008E0
:1000700023010008230100082301000823010008D0
:1000800023010008230100082301000823010008C0
:1000900023010008230100082301000823010008B0
:1000A00023010008230100082301000823010008A0
:1000B000ED190008230100082301000823010008AE
:1000C0002301000823010008230100082301000880
:1000D00023010008A51900082301000823010008D6
:1000E0002301000823010008230100082301000860
:1000F00023010008DFF80CD001F0C0FD00480047E4
:10010000DD160008480400200648804706480047DE
:10011000FEE7FEE7FEE7FEE7FEE7FEE7FEE7FEE7B7
:10012000FEE7FEE753180008F500000832490143D6
:10013000324A1160704770B5002100230F22C47845
:100140001CB32E4C246804F4E064C4F5E064C4F3EA
:100150000721C1F10404E3B20A4144789C40E1B2B2
:100160008478144021430C07210E254C05786155F5
:10017000047804F01F050124AC4005786D11AD0032
:1001800005F1E025C5F8004109E0047804F01F05F9
:100190000124AC401B4D0678761145F8264070BD11
:1001A000194A0A400243154B1B1F1A60704739B1A8
:1001B000124A121D12680243104B1B1D1A6006E002
:1001C0000E4A121D126882430C4B1B1D1A607047A9
:1001D000042808D14FF0E021096941F004014FF0F3
:1001E000E022116107E04FF0E021096921F00401EC
:1001F0004FF0E022116170470000FA050CED00E0BD
:1002000000E400E080E100E080FFFF1F10B504463D
:100210008548844208D10121084600F0BCFA00213B
:10022000012000F0B8FA52E08048844208D1012150
:10023000022000F0B0FA0021022000F0ACFA46E003
:100240007B48844208D10121042000F0A4FA002157
:10025000042000F0A0FA3AE07648844208D1012157
:10026000082000F098FA0021082000F094FA2EE00F
:100270007148844208D10121102000F08CFA00213D
:10028000102000F088FA22E06C48844208D1012155
:10029000402000F080FA0021402000F07CFA16E0B7
:1002A0006748844208D10121802000F074FA0021BF
:1002B000802000F070FA0AE06248844207D10121F0
:1002C000202000F068FA0021202000F064FA10BD20
:1002D000F0B50A4600210023002400BF3DE00125BF
:1002E00005FA01F3156805EA03049C4234D1056858
:1002F0004F000326BE40B543056015794E00B5405A
:100300000668354305601579012D02D01579022D57
:1003100016D185684F000326BE40B54385605579E8
:100320004E00B540866835438560858801268E403D
:10033000B5438580858896798E40B6B235438580F1
:10034000C5684F000326BE40B543C560D5794E0051
:10035000B540C6683543C560491C1029BFD3F0BD00
:100360004FF6FF7101600021017141718171C1710E
:10037000704708B54FF480320092009A0A43009209
:10038000009AC261C161009AC261C2690092C269E9
:10039000009208BD02460020138A0B400BB10120D9
:1003A00000E0002070470146088A7047024600209E
:1003B000938A0B400BB1012000E0002070470146FA
:1003C000888A704701837047418370470AB101836F
:1003D00000E04183704781827047828A4A4082826E
:1003E0007047F0B5002300244D07ED0E02FA05F327
:1003F000CE1000F1200555F826504E07F70E0F26B7
:10040000BE40B543CF1000F1200646F82750CE106D
:1004100000F1200555F8265045EA0304CE1000F1FE
:10042000200545F82640F0BD0000024000040240CF
:1004300000080240000C0240001002400018024078
:10044000001C024000140240F948006840F480702B
:10045000F7490860F64808300068F6490840F44952
:1004600008310860F2480068F3490840F049086024
:100470000846006820F480200860ED4808300068D5
:1004800020F47D00EA49083108600020091D086059
:1004900070470021E64A921C11701146087070479F
:1004A00010B501460022002300204A11012A02D182
:1004B000DF4C236802E0DE4C3434236801F01F0275
:1004C000012494401C400CB1012000E0002010BD2C
:1004D00038B5002000900024002500BF3120FFF730
:1004E000DFFF05460098401C00900098B0F5A06F13
:1004F00001D0002DF2D03120FFF7D2FF08B1012446
:1005000000E00024204638BDC949C91D0870704765
:1005100001460020C64A121D106820F460400843BE
:1005200010607047C5490862704701460020C04A04
:10053000121D106820F4F85040EA01201060704746
:10054000BE49086070470021B94A35321170114622
:1005500008707047BA490860704710B541EA020355
:100560000343B34C0A34237010BDB4490866704786
:10057000B24908677047B2492C310860704740EAB9
:100580000102AB4B0B331A70704701460020A84A9A
:100590000832106820F00300084310607047A44838
:1005A0000830006800F00C00704701460020A04AA7
:1005B0000832106820F0F0000843106070470146D0
:1005C00000209B4A0832106820F4E0600843106065
:1005D000704701460020964A0832106820F46050A7
:1005E00040EAC10010607047F0B5002100220023EE
:1005F0000026002400258E4F08373F6807F00C01C5
:1006000031B1042912D0082913D00C2937D113E0B5
:10061000874F3F1D3F68C7F342356F1C4FF0010CF9
:100620000CFA07FC4FEACC37076036E0854F0760CD
:1006300033E0854F076030E07D4F08373F6807F4AF
:1006400070127B4F08373F6807F440037F4F07EB7A
:1006500092473A78012707EB9353754F08373F6865
:1006600007F480362EB9774F5743B7FBF3F707608F
:1006700004E0754F5743B7FBF3F707600DE06C4F8D
:100680003F1D3F68C7F342356F1C4FF0010C0CFA59
:1006900007FC4FEACC37076000BF00BF644F083744
:1006A0003F6807F0F0010909694F7C5C0768E74083
:1006B00047605F4F08373F6807F4E061090A644FFD
:1006C0007C5C4768E7408760594F08373F6807F40C
:1006D0006051C90A5E4F7C5C4768E740C760F0BD67
:1006E000002100F44032B2F5403F08D1504A116871
:1006F00021F0C04100F0C04211434D4A11604C4A04
:100700003432126822F44032494B34331A601A46AC
:10071000126800F440331A43454B34331A60704773
:10072000474958310860704745495C310860704757
:1007300039B13F4A1C32126802433D4B1C331A60E8
:1007400006E03B4A1C3212688243394B1C331A6064
:10075000704739B1364A203212680243344B203395
:100760001A6006E0324A203212688243304B20334E
:100770001A60704739B12E4A2432126802432C4B5A
:1007800024331A6006E02A4A243212688243284B36
:1007900024331A60704739B1254A10321268024377
:1007A000234B10331A6006E0214A1032126882434C
:1007B0001F4B10331A60704739B11D4A143212684A
:1007C00002431B4B14331A6006E0194A14321268B4
:1007D0008243174B14331A60704739B1144A1832E8
:1007E00012680243124B18331A6006E0104A18329E
:1007F000126882430E4B18331A60704739B10C4AA5
:100800002832126802430A4B28331A6006E0084A6D
:10081000283212688243064B28331A607047C9B1E8
:10082000034A2C3212680243014B2C331A6016E043
:10083000003802400CC0FF88FEFFFEEE0000474279
:10084000800647420024F40000127A0000000020D5
:10085000090000201F4A126882431E4B1A6070472D
:1008600039B11C4A121D126802431A4B1B1D1A6033
:1008700006E0184A121D12688243164B1B1D1A60AF
:10088000704739B1134A1F3A12780243114B1F3B8C
:100890001A7006E00F4A1F3A127882430D4B1F3B35
:1008A0001A7070470B480830006840F080700949A2
:1008B00008310860704701460020064A203A126855
:1008C0000A400AB1012000E00020704701491E39AA
:1008D000087070472C38024010B50446B4F1804FC0
:1008E00008D101210846FFF778FF00210120FFF71A
:1008F00074FF5EE0FB48844208D101210220FFF72B
:100900006CFF00210220FFF768FF52E0F6488442A6
:1009100008D101210420FFF760FF00210420FFF728
:100920005CFF46E0F148844208D101210820FFF72E
:1009300054FF00210820FFF750FF3AE0EC488442C2
:1009400008D101211020FFF748FF00211020FFF7F8
:1009500044FF2EE0E748844208D101212020FFF720
:100960003CFF00212020FFF738FF22E0E2488442CC
:1009700008D101210420FFF71FFF00210420FFF709
:100980001BFF16E0DD48844208D101210820FFF753
:1009900013FF00210820FFF70FFF0AE0D848844228
:1009A00007D101211020FFF707FF00211020FFF7DA
:1009B00003FF10BD00220288B0F1804F08D0C94B60
:1009C000984205D0C84B984202D0C84B984204D1F7
:1009D0004FF68F731A404B881A43C54B984207D085
:1009E000C44B984204D04FF6FF431A400B891A4378
:1009F00002804B68C3620B880385012383827047A2
:100A00004FF0FF314160002101800181418070473A
:100A10000185828270470A46002101884FF68F7354
:100A2000194011430180704741627047C1627047AD
:100A30000146486A70470146088D704721B1028817
:100A400042F00202028004E002884FF6FD731A4071
:100A50000280704721B1028842F00402028004E063
:100A600002884FF6FB731A400280704721B102885A
:100A700042F08002028004E002884FF67F731A4041
:100A80000280704702884FF6F7731A40028002888E
:100A90000A430280704702884FF6FF431A400280E3
:100AA00002880A430280704721B1028842F00102A5
:100AB000028004E002884FF6FE731A4002807047FD
:100AC00030B500230022048C4FF6FE752C400484C0
:100AD000028C038B4FF68F742340AC1E23400C888E
:100AE00023436C1E22400C8922434C8822434C68CD
:100AF00044630383028430BD30B500230022048C9C
:100B00004FF6EF752C400484028C038B48F6FF747B
:100B100023400C884FF6FF7505EA042423434FF663
:100B2000DF7422400C8905EA041422434C8805EA4C
:100B3000041422434C6884630383028430BD30B5BF
:100B400000230022048C4FF6FF652C400484028CA5
:100B5000838B4FF68F7423400C8823434FF6FF544A
:100B600022400C894FF6FF7505EA042422434C8885
:100B700005EA042422434C68C4638383028430BDA5
:100B800030B500230022048C4EF6FF752C400484FF
:100B9000028C838B48F6FF7423400C884FF6FF7558
:100BA00005EA042423434DF6FF7422400C8905EA2C
:100BB000043422434C8805EA043422434C6804641C
:100BC0008383028430BD0021018041804160018126
:100BD000704770B5034600200024184618300125E0
:100BE0008D40ACB21D8CA5431D8409B1082909D1E3
:100BF00000EB6100056825F0700505600568154388
:100C000005600EE00D1FC5F34E052844056825F468
:100C1000E045056005684FF6FF7606EA0226354393
:100C2000056070BD4163704781637047C163704761
:100C3000016470470A460021018B4FF68F731940FB
:100C40001143018370470A460021018B48F6FF7368
:100C500019404FF6FF7303EA0223194301837047DB
:100C60000A460021818B4FF68F731940114381830F
:100C700070470A460021818B48F6FF7319404FF6F2
:100C8000FF7303EA02231943818370470A46002158
:100C9000018B4FF6F77319401143018370470A46E1
:100CA0000021018B4FF2FF7319404FF6FF7303EAE7
:100CB00002231943018370470A460021818B4FF6B6
:100CC000F77319401143818370470A460021818BD5
:100CD0004FF2FF7319404FF6FF7303EA02231943E3
:100CE000818370470004004000080040000C004071
:100CF000001000400014004000080140000C0140BA
:100D0000001001400A460021018B4FF6FB73194089
:100D10001143018370470A460021018B4FF6FF33D0
:100D200019404FF6FF7303EA02231943018370470A
:100D30000A460021818B4FF6FB73194011438183D2
:100D400070470A460021818B4FF6FF3319404FF65A
:100D5000FF7303EA02231943818370470A46002187
:100D6000018B4FF67F7319401143018370470A4688
:100D70000021018BC1F30E014FF6FF7303EA02233A
:100D80001943018370470A460021818B4FF67F7318
:100D900019401143818370470A460021818BC1F3BA
:100DA0000E014FF6FF7303EA022319438183704754
:100DB0000A460021018C4FF6FD731940114301844E
:100DC00070470A460021018C4FF6DF7319404FF639
:100DD000FF7303EA02131943018470470A46002196
:100DE000018C4FF6FF5319404FF6FF7303EA0223BD
:100DF0001943018470470A460021018C4DF6FF73A8
:100E000019404FF6FF7303EA023319430184704718
:100E100002894FF6F7731A40028102890A43028160
:100E2000704730B5002301248C40A3B2048C9C434E
:100E30000484048C02FA01F5ADB22C43048430BD65
:100E4000828B4FF2FF331A408283828B4FF6FF73FF
:100E500003EA01231A4382837047F0B50C46154616
:100E6000002100220026078C4EF6FF7C07EA0C07C3
:100E70000784818B028C4FF6FF7707EA043640F631
:100E8000FF4739404FF6FF7707EA052739434FF60A
:100E9000FF7707EA0337394345F6FF773A4046F4D0
:100EA00080573A4381830284F0BD828B4FF6F373FF
:100EB0001A408283828B0A4382837047F0B50C46C6
:100EC0001546002100220026078C4FF6FF6C07EA2A
:100ED0000C070784818B028C4FF6FF7707EA042604
:100EE0004FF60C7739404FF6FF7707EA03172F4389
:100EF00039434FF2FF573A4046F480773A438183B3
:100F00000284F0BD028B4FF2FF331A400283028B42
:100F10004FF6FF7303EA01231A4302837047F0B5CB
:100F20000C461546002100220026078C4FF6EF7C68
:100F300007EA0C070784018B028C4FF6FF7707EA5C
:100F4000041640F6FF4739404FF6FF7707EA0337AC
:100F500039434FF6FF7707EA052739434FF65F77A6
:100F60003A4046F010073A4301830284F0BD028BF9
:100F70004FF6F3731A400283028B0A4302837047D1
:100F8000F0B50C46154600210022068C4FF6FE7780
:100F90003E400684018B028C4FF60C7631407E1C5D
:100FA00006EA03162E4331434FF6F576324044F0FD
:100FB0000106324301830284F0BD70B505460C463C
:100FC000208850B92389A28861882846FFF7D8FF76
:100FD000E1882846FFF7CBFF25E0208804280AD1C6
:100FE0002389A28861882846FFF799FFE18828466F
:100FF000FFF788FF17E0208808280AD12389A288F4
:1010000061882846FFF75AFFE1882846FFF74DFF21
:1010100009E02389A28861882846FFF71EFFE1883E
:101020002846FFF70DFF70BD00210180418001219E
:1010300081800021C180018170472DE9F041054682
:101040000C4600260127608808B9022600E0002629
:10105000A088012801D1022700E001272088A0B93B
:101060002389A28861882846FFF78AFFE1882846FD
:10107000FFF77DFF23893A4631462846FFF74FFFA9
:10108000E1882846FFF73EFF13E02389A2886188A4
:101090002846FFF744FFE1882846FFF733FF2389FE
:1010A0003A4631462846FFF76BFFE1882846FFF7AE
:1010B0005EFFBDE8F0810146486B70470146886BD2
:1010C00070470146C86B70470146086C70471AB1FB
:1010D00083890B43838102E083898B43838170473B
:1010E0008182704702460020138A0B400BB1012019
:1010F00000E000207047CA430282704730B50246C4
:10110000002000230024158A05EA0103958905EAD9
:10111000010413B10CB1012000E0002030BDCA432E
:101120000282704741EA0203A0F8483070471AB1C2
:1011300083890B43838102E083898B4383817047DA
:1011400021B1828842F00802828004E082884FF652
:10115000F7731A408280704701894FF6F872114088
:10116000018170470A46002101894FF68F731940AB
:1011700011430181704730B504460D46294620468B
:10118000FFF7F0FF208940F00700208130BD2DE9F6
:10119000F04104460D4616461F46602D06D13B46DB
:1011A000012231462046FFF7BAFE05E03B46012208
:1011B00031462046FFF7E4FE29462046FFF7D2FFDE
:1011C000208940F007002081BDE8F08130B50C4651
:1011D00000210189C9B24FF6FF7505EA03251543C1
:1011E00025432943018130BD2DE9F04105460E46D6
:1011F00017469846002443463A4631462846FFF7AC
:10120000E5FF2C894FF6F870044044F007044FF6D0
:101210008F70044044F070042C81BDE8F081F0B57B
:1012200004460D4616461F463B4632462946204692
:10123000FFF7CCFF208940F480402081F0BD8288F8
:101240004FF68F731A40828082880A4382807047EB
:1012500002894FF6F8731A40028102890A4302811B
:10126000704702894FF67F731A40028102890A4350
:1012700002817047F0B50C4615461E46002100223B
:1012800000230189028B038C4FF6F8773940214304
:101290004FF6FC473A4040F201173A434FF6DD77EC
:1012A0003B404FF6FF7707EA06172F433B43018188
:1012B00002830384F0BD21B1828842F080028280E3
:1012C00004E082884FF67F731A408280704730F8BE
:1012D000502F02EA1142028002888BB21A4320F892
:1012E0005029704710B50446F748844209D10121BE
:1012F0008803FFF761FA00214FF48040FFF75CFAA2
:1013000032E0F248844209D101214804FFF765FA2E
:1013100000214FF40030FFF760FA25E0EC488442EA
:1013200009D101218804FFF758FA00214FF48020E9
:10133000FFF753FA18E0E748844209D10121C804B5
:10134000FFF74BFA00214FF40020FFF746FA0BE0BD
:10135000E148844208D101210805FFF73EFA002147
:101360004FF48010FFF739FA10BD2DE9FF4705460D
:101370000E460024A14600BFA046B08900B100BFC0
:101380002C8A24F44054F08804432C82AC8941F226
:101390000C608443B0883189084371890843044351
:1013A000AC81AC8A24F44074B0890443AC826846B2
:1013B000FFF71AF9C448854202D1DDF80C9001E02C
:1013C000DDF80890A88900F4004040B109EBC9009D
:1013D00000EB091031684900B0FBF1F707E009EBB9
:1013E000C90000EB091031688900B0FBF1F76420F7
:1013F000B7FBF0F004012009642101FB1078A889F3
:1014000000F4004040B1322000EBC800B0FBF1F026
:1014100000F00700044308E0322000EB08106421CC
:10142000B0FBF1F000F00F0004432C81BDE8FF8712
:101430004FF41651016000218180C18001810C218F
:10144000418100218181704710B502460020108A39
:1014500020F470600B884C8823438C882343CC880D
:1014600023431843108210BD0021018041808180F8
:10147000C180704721B1828942F40052828104E028
:1014800082894DF6FF731A4082817047028B02F405
:101490007F420283028B0A430283704721B1828913
:1014A00042F40042828103E08289C2F30E0282810B
:1014B000704721B1828A42F40062828204E0828A0B
:1014C0004FF2FF731A4082827047C1F30802828094
:1014D000704701468888C0F308007047028A4FF6BB
:1014E000F0731A400282028A0A430282704721B1D5
:1014F000828942F00202828104E082894FF6FD7304
:101500001A408281704782894FF2FF731A408281AC
:1015100082890A4382817047028A4FF6DF731A403C
:101520000282028A0A430282704721B1028A42F48F
:101530008042028204E0028A4BF6FF731A40028264
:101540007047818941F001018181704721B1828A10
:1015500042F00802828204E0828A4FF6F7731A4052
:1015600082827047028BD2B20283028B42EA01224E
:101570000283704721B1828A42F02002828204E015
:10158000828A4FF6DF731A408282704721B1828AC5
:1015900042F01002828204E0828A4FF6EF731A4012
:1015A00082827047828A4FF6FB731A408282828A57
:1015B0000A438282704721B1828A42F0020282820B
:1015C00004E0828A4FF6FD731A40828270471AB196
:1015D000838A0B43838202E0838A8B438382704732
:1015E000F0B50346002400260025002040F66A17C7
:1015F000B94200D100BF1846C1F3421401F01F06E2
:10160000012707FA06F5012C01D10C3004E0022C69
:1016100001D1103000E014301AB107682F43076081
:1016200002E00768AF430760F0BD02460020B1F555
:10163000007F00D100BF13880B400BB1012000E0F8
:101640000020704701F40072B2F5007F00D100BFA6
:10165000CA430280704770B502460024002300256B
:10166000002040F66A16B14200D100BFC1F3421516
:1016700001F01F03012606FA03F3012D02D196891A
:10168000334006E0022D02D1168A334001E0968AEB
:1016900033400C12012606FA04F41688344013B1C4
:1016A0000CB1012000E0002070BD10B50022002325
:1016B00040F66A14A14200D100BF0A1201249440EE
:1016C000A3B2DC43048010BD003801400044004058
:1016D00000480040004C00400050004086B01422FA
:1016E00012A101A800F0B7FA00F0AAFA132201A98A
:1016F000134800F019FA13A000F0D2FA15E0002008
:1017000000F001FA4FF4FA7000F0C2F94FF4FA70E9
:1017100000F0BEF9012000F0F6F94FF4FA7000F085
:10172000B7F94FF4FA7000F0B3F9E8E748656C6C6C
:101730006F2053544D33324C313531210D0A0000A6
:1017400000380140B4AEBFDA31B2E2CAD40A0000B8
:101750000CB50020019000908748006840F480306C
:101760008549086000BF8448006800F4003000909C
:101770000198401C0190009818B90198B0F5A06F2D
:10178000F1D17D48006800F4003010B101200090D4
:1017900001E0002000900098012859D177480068A6
:1017A00040F00400754908600846006840F00200F7
:1017B00008600846006840F0010008606E48243068
:1017C000006840F080506C4924310860C8146C49AE
:1017D000086000BF6A48406800F010000028F9D196
:1017E00065480830006864490831086008460068A8
:1017F00008600846006808600846006820F47D001C
:1018000008600846006840F49A0008605A4800687A
:1018100040F080705849086000BF5748006800F0E9
:1018200000700028F9D054480830006820F0030008
:101830005149083108600846006840F0030008601C
:1018400000BF4D480830006800F00C000C28F8D1AB
:101850000CBD10B54848006840F4807046490860E7
:101860004548083000684749084043490831086046
:1018700041480068444908403F49086008460068FC
:1018800020F4802008603C480830006820F47D0087
:101890003949083108600020091D0860FFF758FF2A
:1018A0004FF000603949086010BD70B5002200207B
:1018B000002100240023304D08352D6805F00C026E
:1018C00032B1042A10D0082A12D00C2A39D113E0E0
:1018D000294D2D1D2D68C5F342335D1C0126AE40F8
:1018E000F5032B4E356038E02A4D294E356034E043
:1018F000294D274E356030E01F4D08352D6805F421
:1019000070101D4D08352D6805F44001234D05EB81
:1019100090452878012505EB9151174D08352D6824
:1019200005F4803434B91B4D4543B5FBF1F5184E31
:10193000356005E0184D4543B5FBF1F5144E3560B3
:101940000BE00D4D2D1D2D68C5F342335D1C0126A6
:10195000AE40F5030E4E356000BF00BF064D0835A2
:101960002D68C5F303150E4E725D094D2D68D540E7
:10197000074E356070BD000000380240003C024058
:10198000007000400CC0FF88FEFFFEEE08ED00E096
:101990001C0000200024F40000127A002000002027
:1019A0002900002010B540F225511B48FFF753FED7
:1019B00070B11948FFF78DFDC4B221461648FFF7F4
:1019C00084FD00BF80211448FFF72FFE0028F9D0C6
:1019D00010BD704700BFFEE700BFFEE700BFFEE797
:1019E00000BFFEE7704770477047704710B5012190
:1019F0008807FFF783FB70B101218807FFF78FFB92
:101A000006480078401C05490870084600780528FB
:101A100001D10020087010BD003801403A000020BC
:101A20004FF0E021096921F004014FF0E02211613B
:101A3000C21700EB5272C2F3C702234B1A70194649
:101A4000097801EB4102C2EBC1114FF6FF7202EAC5
:101A5000C1011E4A1180704701461B4A12784A4351
:101A60004FF0E0235A6100229A6101221A6100BFFF
:101A70004FF0E022106900F001021AB100F4803248
:101A8000002AF5D000224FF0E0231A619A617047D6
:101A900001460E4A12884A434FF0E0235A61002261
:101AA0009A6101221A6100BF4FF0E022106900F034
:101AB00001021AB100F48032002AF5D000224FF062
:101AC000E0231A619A6170473E0000204000002028
:101AD0001CB501210846FEF72BFE01208DF80400FD
:101AE00000208DF8060001208DF8070002208DF8F7
:101AF0000500009069460B48FEF7EAFB0221094801
:101B0000FEF760FC1CBD30B10649898A41F0020134
:101B1000044A918205E00349898A21F00201014AC1
:101B200091827047000002402DE9F04107460D46C2
:101B3000164600240CE0295D3846FFF7C6FC00BFBE
:101B400040213846FFF771FD0028F9D0601C84B2AF
:101B5000B442F0DBBDE8F08170B504460D46E1B259
:101B60003548FFF7B2FC00BF80213348FFF75DFD29
:101B70000028F9D0204670BD10B588B00446012178
:101B80008803FEF7E6FD01210846FEF7D1FD2A484D
:101B9000FFF7A8FB4FF4C060029002208DF80C0004
:101BA0008DF80D0000208DF80E0001208DF80F003B
:101BB00002A92248FEF78CFB4FF48060029002A934
:101BC0001E48FEF785FB072209211C48FEF709FC89
:101BD00007220A211948FEF704FC04940020ADF8FE
:101BE0001400ADF81600ADF81800ADF81C000C207C
:101BF000ADF81A0004A91048FFF7B7FB01210E4801
:101C0000FFF738FC012240F225510B48FFF7E8FCB2
:101C100025208DF8040003208DF805008DF80600BE
:101C200001208DF8070001A8FEF785FA402102483F
:101C3000FFF708FD08B010BD003801400000024069
:101C400010B52020FFF7ECFEFFF742FF4FF41650CF
:101C5000FFF792FF10BD40EA01039B0703D009E0A4
:101C600008C9121F08C0042AFAD203E011F8013B88
:101C700000F8013B521EF9D270470000064C074D98
:101C800006E0E06840F0010394E80700984710344C
:101C9000AC42F6D3FEF732FAF01C0008101D000823
:101CA000014A024900F013B8591B00084400002003
:101CB00002E008C8121F08C1002AFAD17047704715
:101CC000002001E001C1121F002AFBD170472DE95D
:101CD000F04116460F460446002503E03946B0475A
:101CE000641C6D1C20780028F8D12846BDE8F081DE
:101CF000101D00080000002048000000B01C000873
:101D0000581D00084800002000040000C01C000806
:101D1000030406080C101820300000000001020324
:101D20000401020304060708090000000048E80156
:101D3000030406080C10182030000000000000000A
:101D4000000102030406070809000000000000006B
:081D500000000000000000008B
:04000005080000F5FA
:00000001FF
